:100000002500A10B0802E201000800080008000812
:10001000030814082C0847086008770827085A08BE
:100020007D089508A808B608C108C908D008D608F0
:10003000DA08DE08E208E508E708E908EB08ED0859
:10004000EE08EF08F008F108F208F3080802E201F0
:10005000000800080008000884080D0806080408C5
:100060000308020801080108010801080108010845
:100070000108010801080108010801080108010838
:100080000108010801080108010801080108010828
:1000900001080108090C2E00400003042F000F0383
:1000A0002D030306CC01EE024E0A2C002C032D0377
:1000B0002C032D032C032D032C032D030008040017
:1000C000FF0C2D002E002F00090C24000B0C3D000E
:1000D000470400008F094706740AAF096606C70582
:1000E0000000670646040000FC0C3F024306860A37
:1000F000FF017F00FD02810A0306FE0ABD02000027
:10010000680A000000000307680AF30B0000000003
:100110000000C706BF02C704FE03680AB20B6607E9
:100120000008BF027E004705AF0966070008BF024E
:100130000000A706A30A0209290026093000470487
:10014000DF038F0AB20B0000000000000000000077
:100150000000000000000000000000009F0AC10332
:10016000C10A09029C004306DC0A0306BA0ABC0263
:100170001202BD0AFC00130287052100080C0600CC
:100180000008E707E50AE70440000706080D060631
:10019000020D2606040DE2010605000826050008EA
:1001A00026040008060400082605000806040008C6
:1001B0000605000826040008870400000000090264
:1001C0004307F40A0B0C06000008FA03EF0ADC00F0
:1001D0003A00FB02F30A10023B00E70500081C028C
:1001E000890138007802000000000008100C84002B
:1001F000070E4306EF0BC706BF02010B090C3D00BB
:10020000A4024704C7048F0947060D0BAF09660611
:10021000C7050000000000000000FC0C3F02430680
:10022000F60AFF017F00FD02370B0306FE0A0A02F1
:100230008B018C018D018E018F014307D90B6A025E
:100240006B026C026D026E02AF09E400A3054F0A57
:100250001C029A0003071A02F80E4306310BA3058D
:100260004F0A060C3D00FD02330BAF09280B670651
:1002700046056003010B010C3100FF0C3600000C39
:10028000370088061602590B110296002C00030451
:100290002C03180CEC01030C88002D004A09090CF2
:1002A000AD0011020307410B00000000CD01030661
:1002B000160229006B0017024306940B7F0E2A00DA
:1002C000F707650B040C8800680B48021F0E00003E
:1002D0002E008E076E06830B2F004306740B03045B
:1002E0002A032B03EE02700B4F02070E2E0043066B
:1002F0007D0B00000000EE02790B17027F0E2F002D
:100300000A028F00940B8A03070ECA012C00070C07
:100310008E002D004A090D022F002C032D032C0303
:100320002D03CD008F008A00F7079D0BC90103073D
:1003300029000000A705A4045F0A8900030629001C
:100340009A0BD70C0200580289019C014307AB0BA2
:10035000080C06005F0A7C00690068007E007F00D0
:100360007A00BA020B0C06006600300C24006A000A
:10037000A3050509A3044306B80B0F0220003F0C98
:1003800084013F0E4306C70BA402AA02B80B120257
:100390004306010DFF0FA4043200A4051302430617
:1003A000010DFF0F7500A4043300090C24005F0A3F
:1003B00000000000000000000000AF090000000085
:1003C00000000000000000000000000000005F0AC4
:1003D000000000000000000000000000000000001D
:0A03E0000000000000000000D80B30
:10040000840C2700310A800C060A830C2700A00CFC
:10041000C6042900080C2800E6046903C604030684
:10042000C6050000E605E8020C0A0000E60400002C
:10043000C60500000000E605C606E704E604E70777
:10044000470A07020F0EE2012B0A2E0A470A2B0A5F
:10045000310A360A470AA7020A02090AA7020F024E
:10046000090AE605C605A702A10C080AC605000090
:10047000E605080C2800E6050305C60703046F031C
:10048000E604C605E8023B0AE6050000E604C604E9
:10049000E6054A0A4B0AC605E70700080108A40555
:1004A0000A02EA076B0A98014307650A0B029901E1
:1004B0004307650A2C0C2400B407650A2706650A61
:1004C0007B0A640A2706FA0B770A0A02F00E700FFD
:1004D0004306FB0AFA0B4306610AB4079001430680
:1004E000620A1A027F0E2704430727058A01430781
:1004F000650A2B0C240080032F000F03070EE20176
:10050000A70ADA0B870B8F0B630B7E0BFA0B460BDC
:100510002400070C4C019E098C07950A6C062001EB
:10052000FF0F6C07600104020D0B400143069B0A9C
:100530006C06300BFA0B6C07300BFA0BE20101086A
:100540000208040808081008200840088008A006CF
:10055000CC0B0003070EE201AE0BD90BFA0BB70B65
:10056000FA0BBE0BFA0BC50B3C02430700088007D1
:10057000C50A0706C00A5406C20A8605A604000872
:100580005406BD0A8604A60500088604A6040008D1
:1005900047046704000F43063008010F4306310883
:1005A000030F43063208010F43063308070F4306C3
:1005B0003608010F43063708150F43063808010FA8
:1005C00043063908030F43063A080E0F4306340862
:1005D0002C0F43063B08010F43063C08030F43065C
:1005E0003D086705340F43064008010F43060D0818
:1005F00067044705FF0804020F0E0C0F4307460B64
:100600000B02C8094706FA0B67066A07090B350093
:10061000350C4A07880A6A07250B0F0E2A000509C0
:1006200000028F014306A3044306B50B00022F000E
:10063000D4061C0BD405FC0B030943061C0BA304B6
:10064000B50B0A0220004000280B6706440B0F0E72
:100650002A00050900028F014307A30443075F0A2C
:10066000C306340BC305FC0B080C0600060C2E0059
:100670006F000400EF033A0BEE02380B0B0C060080
:10068000C304A404A3045F0A80012C0B0B02F90F1E
:100690004306210B0A027D0F43065D0B010F430643
:1006A0005A0B0A02070ED501C8094706FA0B6A075A
:1006B000250B0D0B0A02070E570BEB0003046B030F
:1006C0004B033500FA0B800634053406B4099B064B
:1006D000FA0B8706DB07750B0706720B5406740BC3
:1006E000A605750B5406700B860500020F0E5B0104
:1006F0004306830BBB0667054605FA0B8007FA0B1A
:100700009B07FA0B690BBB0667044604FA0B140639
:10071000910BFA06930B0707970B0704AE0B140611
:10072000890BFA068B0B0706970B0705AE0BA70480
:1007300040031E0E2800800608053407080434070D
:10074000B40908024306B50BFD0E4306AE0B940632
:10075000FA0BA304440BA304A404A10B060426046F
:10076000A4047A00BA027C006F006900FA0B7404DA
:1007700003077405340C200014020D0BB4040307A6
:10078000B405340C200014020D0B54040307540567
:10079000340C200014020D0B0C023A000002120F60
:1007A0004306FA04010F4306FA053A0C20001A0228
:1007B0000D0BFA0B00023F0F4307FA0BA402E006F1
:1007C000E90B1406EB0BFA06ED0B0707F10B070418
:1007D000AE0B1406E30BFA06E50B0706F10B070553
:1007E000AE0B00032F000F0328004003290034053F
:1007F000A705FA0BD404C304A304A4045F0A800C65
:021FFE00E60FEC
:00000001FF
